:103800000C943E1C0C94481C0C94481C0C94481CB2
:103810000C94481C0C94481C0C94481C0C94481C98
:103820000C94481C0C94481C0C94481C0C94481C88
:103830000C94481C0C94481C0C94481C0C94481C78
:103840000C94481C0C94481C0C94481C0C94481C68
:103850000C94481C0C94481C0C94481C0C94481C58
:103860000C94481C0C94481C0C94481C0C94481C48
:103870000C94481C0C94481C0C94481C11241FBE2A
:10388000CFEFD4E0DEBFCDBF0E94301D0C94EF1E01
:103890000C94001C9FEF92B911B887E585B988EAAE
:1038A00084B998B98CE387B98DE08BB982EF8AB976
:1038B00008950F931F93CF93DF938C01EA01653432
:1038C00079F48881998181BD92BD0196998388831D
:1038D000F89A80B50E94DC1E0150104091F721C07B
:1038E0006634F9F488819981880F991F99838883B8
:1038F000E881F981E4918E2F0E94DC1EE881F98134
:103900003196E4918E2F0E94DC1E88819981029667
:10391000998388830250104059F79695879599832B
:103920008883DF91CF911F910F9108957F928F929D
:103930009F92AF92BF92CF92DF92EF92FF920F933E
:103940001F93DF93CF93CDB7DEB7C058D0400FB6EB
:10395000F894DEBF0FBECDBF4C015A01653461F54E
:103960007E010894E11CF11C67018E0C9F1C05C0B0
:103970000E94E81ED6018D936D01C814D904C1F7C9
:1039800007B600FCFDCF14C0F5012081318121BDB7
:1039900032BDD7018C9180BDFA9AF99AF999FECF80
:1039A0002F5F3F4FF501318320830894E11CF11C08
:1039B000EC14FD0449F73EC0663411F08FE33BC0C0
:1039C000DA01CD90DC901197CC0CDD1CCD92DC920D
:1039D000772473940E94E81E082F10E00E94E81ECE
:1039E000D501ED91FC91F82EEE240E291F29080136
:1039F00070925700E89511249F012E5F3F4FF5010B
:103A0000318320838EEF9FEF880E991E81149104DD
:103A100009F785E0F60180935700E89507B600FCAA
:103A2000FDCF81E180935700E89536952795D50124
:103A30002D933C938DE0C058DF4F0FB6F894DEBF56
:103A40000FBECDBFCF91DF911F910F91FF90EF90EF
:103A5000DF90CF90BF90AF909F908F907F90089510
:103A60002F923F924F925F926F927F928F929F928E
:103A7000AF92BF92CF92DF92EF92FF920F931F937C
:103A8000DF93CF9300D0CDB7DEB70E944A1C179AC0
:103A90000E94D51E079968C18BED88B909E013E033
:103AA000212E312C2E010894411C511C0E94E81E2D
:103AB000982F813611F489E554C1813459F40E945C
:103AC000E81E182F0E94E81ED12ECC2490E08C29ED
:103AD0009D2980C0853699F4E0E0F0E009C007B682
:103AE00000FCFDCF23E020935700E895E058FF4FFE
:103AF00088E3E030F80798F3FA83E98305C182365A
:103B000041F489E50E94DC1E80E00E94DC1E80E812
:103B100028C1823499F40E94E81E182F0E94E81EE2
:103B2000B12EAA24E82EFF24EA28FB280E94E81ED2
:103B3000682FC701A2010E94961C13C1873699F411
:103B40000E94E81E182F0E94E81E912E8824E82E5D
:103B5000FF24E828F9280E94E81E682FC701A20167
:103B60000E94591CA3CF8235B9F407B600FCFDCFE3
:103B7000E1E1E0935700E895E981FA81EE0FFF1F3C
:103B80003196E4918E2F0E94DC1EE981FA81EE0FBE
:103B9000FF1FE4918E2F52C0833629F40E94E81E45
:103BA000E82EFF24B1C08334C1F40E94E81E782EB1
:103BB0006624E628F72807B600FCFDCF89819A81A4
:103BC000FC01EE0FFF1F21E0070120935700E8954D
:103BD000112401969A83898397C08D36A1F4E981D7
:103BE000FA818CE1E030F80720F08FE30E94DC1EC0
:103BF0008BC007B600FCFDCFEE0FFF1F25E0209322
:103C00005700E89581C0843489F407B600FCFDCFE5
:103C100089819A8181BD92BD0E94E81E80BDFA9A79
:103C2000F99AF999FECF89819A81D3CF843671F4BC
:103C300089819A8181BD92BDF89A80B50E94DC1E6F
:103C400089819A8101969A83898330CF8C3661F479
:103C500007B600FCFDCF0E94E81EE1E0F0E0082E70
:103C600000935700E89550C0823749F407B600FC2E
:103C7000FDCFE1E0F0E000935700849172C08634FC
:103C800059F487B790E0FC01E170F07080FDF9CF46
:103C900000935700849165C08E3441F407B600FC50
:103CA000FDCFF1010093570084915BC0813549F449
:103CB00007B600FCFDCFE2E0F0E0009357008491EE
:103CC00050C0803509F18C34F9F0853471F407B6B1
:103CD00000FCFDCFF1E1F0935700E8958DE00E94E4
:103CE000DC1EE0E0F0E00995E1CE803711F483E5D9
:103CF00038C0843711F480E034C08857823010F027
:103D0000943521F40E94E81E8DE02BC09335A1F478
:103D100081E40E94DC1E86E50E94DC1E82E50E9492
:103D2000DC1E82E40E94DC1E8FE40E94DC1E8FE415
:103D30000E94DC1E84E515C0963529F481E30E94BB
:103D4000DC1E85E30EC0933741F48AE00E94DC1E3E
:103D500084E90E94DC1E8EE104C09B3109F4A6CEEA
:103D60008FE30E94DC1EA2CE07B600FCFDCF81E1EE
:103D700080935700E8958FEF88B9E0E0F0E009956F
:103D80000F900F90CF91DF911F910F91FF90EF90C7
:103D9000DF90CF90BF90AF909F908F907F906F906B
:103DA0005F904F903F902F90089589E18093C400D9
:103DB00088E18093C10008958093C6008091C0007F
:103DC00086FFFCCF8091C00080648093C00008957E
:103DD0008091C00087FFFCCF8091C6000895F894C1
:023DE000FFCF13
:0400000300003800C1
:00000001FF
